:0200000030C10D
:10000200FECFFDCFFCCFFBCFFACFF9CFF8CF6DC338
:1000120060C3F5CFF4CFF3CFF2CFF1CFF0CFEFCF74
:10002200EECFEDCF000000000000002F000000071F
:10003200000700147F147F14242A7F2A12C4C810D8
:10004200264636495522500005030000001C224175
:10005200000041221C0014083E081408083E08084B
:1000620000005030001010101010006060000020DE
:10007200100804023E5149453E00427F4000426161
:100082005149462141454B311814127F10274545ED
:1000920045393C4A49493001710905033649494904
:1000A20036064949291E0036360000005636000041
:1000B20008142241001414141414004122140802DA
:1000C20001510906324959513E7E1111117E7F4973
:1000D2004949363E414141227F4141221C7F4949E3
:1000E20049417F090909013E4149497A7F080808C7
:1000F2007F00417F41002040413F017F081422419F
:100102007F404040407F020C027F7F0408107F3E08
:100112004141413E7F090909063E4151215E7F0965
:10012200192946464949493101017F01013F4040B1
:10013200403F1F2040201F3F4038403F63140814B7
:100142006307087008076151494543007F41410038
:10015200552A552A550041417F00040201020440FC
:1001620040404040000102040020545454787F482B
:100172004444383844444420384444487F38545432
:100182005418087E0901020C5252523E7F080404A0
:100192007800447D40002040443D007F1028440008
:1001A20000417F40007C041804787C0804047838FD
:1001B200444444387C14141408081414187C7C0831
:1001C2000404084854545420043F4440203C404016
:1001D200207C1C2040201C3C4030403C44281028FD
:1001E200440C5050503C4464544C44000000000005
:1001F2004C4346004D65746572006B68617A616DAF
:10020200612E636F6D00202020202020006E4800A8
:100212007548006D4800204800576169742E2E2EE3
:10022200006E4600704600487A004C204D657465A9
:10023200720043204D657465720046204D657465F9
:100242007200446F6E652E2E2E0001002D4E414E1F
:10025200000003000500EE0101005F034C020000F4
:10026200F894EE27ECBBF1E0FBBFEBBFE5BFF8E192
:10027200F1BDE1BD8DE0A2E0BB27ED938A95E9F7E0
:1002820080E094E0A0E6ED930197E9F7E4E5F2E07F
:1002920085919591009761F0A591B5910590159082
:1002A200BF01F00105900D920197E1F7FB01F0CF3C
:1002B200EFE5EDBFE4E0EEBFC0E6D1E098C2E4ECCA
:1002C200E2BBE3E0E1BBE0E0E5BBE0E2E4BBE1E0AE
:1002D200E3BFE0E0E2BFEFBDEEBDEDBDECBDE7BDCB
:1002E200E6BDEBBDEABDE9BDE8BDE5E0E9BF0895C5
:1002F200C49AE7B3EF63E7BBC19AE0D1C498DED1F9
:10030200C49AE0E5EDB9C29AE1E2EA93E0E0EA9349
:10031200C5D1E8ECEA93E0E0EA93C0D1E6E0EA93E3
:10032200E0E0EA93BBD1E3E1EA93E0E0EA93B6D1FD
:10033200E0E2EA93E0E0EA93B1D1ECE0EA93E0E0B4
:10034200EA93ACD1E8EFF1E0E0935A03F0935B0358
:10035200E0E0F0E0E0935C03F0935D0301D006C2BD
:1003620082D900E010E0083FE1E01E074CF4A0E66D
:10037200B1E0A00FB11FE0E0EC930F5F1F4FF3CF8E
:10038200E0E0F0E0E0935A03F0935B03E7EFF1E083
:10039200E0935C03F0935D03E1E0E0935E0312C23D
:1003A200E981F0E03197A6E0B0E032D7BF01E88101
:1003B200F0E03197A4E5B0E02BD7E60FF71FE0930A
:1003C2005803F093590378C14AD9E0915A03F09146
:1003D2005B03A0915803B0915903AE17BF0744F4D1
:1003E200E0915803F0915903E0935A03F0935B03B1
:1003F200AE81A03210F0AC3710F0ECE5EE83AF81A5
:10040200A13009F510E01530E8F4A8E5B3E0ED916C
:10041200FD913196FE93EE933197E05AFE4FBF0164
:10042200EE81E052A5E0EA9FF001EA5DFF4FDF01B5
:10043200E12FF0E0EA0FFB1FE491EE0FDB01EC93FA
:100442001F5FE1CF7DC0AF81A23009F079C0E0919A
:100452005803F0915903E455F040AF01E0915A037B
:10046200F0915B034E175F0724F440935A035093B5
:100472005B0355230AF483C010E0153008F057C01F
:10048200EE81E052A5E0EA9FF001EA5DFF4FDF0155
:10049200E12FF0E0EA0FFB1FE491EE0F0E2FE02FA9
:1004A200E170A3E0EA9FF0013E2FE02FE270A6E0A8
:1004B200EA9FF0013E2BE02FE470ACE0EA9FF001EE
:1004C2003E2BE02FE870A8E1EA9FF0013E2B029557
:1004D2000F70E02FE170A3E0EA9FF0012E2FE02FD2
:1004E200E270A6E0EA9FF0012E2BE02FE470ACE070
:1004F200EA9FF0012E2BE02FE870A8E1EA9FF001BD
:100502002E2BFA014F5F5F4FE05AFE4F3083FA0104
:100512004F5F5F4FE05AFE4F3083FA01EE54FE4FB9
:100522002083FA01ED54FE4F20831F5FA6CFE09196
:100532005803F09159033B96E0935803F093590303
:10054200E0915C03F0915D03A0915803B0915903CF
:10055200EA17FB0744F4E0915803F0915903E09342
:100562005C03F0935D03A8E5B3E0ED91FD91319654
:10057200FE93EE933197E05AFE4FA0E0A08376D827
:1005820028960895E881F981E491E03061F0EA81EA
:10059200EA93E981FA813196E983FA833197E4910A
:1005A200EA9312DFEFCF0FC0A881B981EC91E0305E
:1005B20051F0EA81EA93A981BA81ED91A983BA83C4
:1005C200EA9302DFF1CF239608954DD8A0915B0301
:1005D200AA231AF4E0E0F0E00AC0A0915A03B09115
:1005E2005B03A83FE1E0BE0734F0E7EFF1E0E09300
:1005F2005A03F0935B03A0915D03AA231AF4E0E08F
:10060200F0E00AC0A0915C03B0915D03A83FE1E075
:10061200BE0734F0E7EFF1E0E0935C03F0935D0393
:10062200A0915A03B0915B03E4E5F0E00ED6E068D6
:10063200EA93E0E0EA9332D0A0915A03B0915B03CF
:10064200E4E5F0E0FDD5E064EA93E0E0EA9326D049
:1006520000915A0310915B03E0915C03F0915D03FA
:10066200E017F10764F0A0E6B1E0A00FB11FEC9132
:10067200EA93E1E0EA9312D00F5F1F4FEDCFE7EF6D
:10068200F1E0E0935A03F0935B03E0E0F0E0E093E3
:100692005C03F0935D03E0935E0394C0C298A8816B
:1006A200A13011F4C09A01C0C098E981EFB9EEB14E
:1006B200E078E038E1F7C29A22960895D4D700E0B4
:1006C20013E80030EDE71E071CF40F5F1F4FF9CF50
:1006D20079C0EA93FA93EFB7EA93F30131963F01B7
:1006E200E991EFBFF991E9911895EA93EFB7539425
:1006F200EFBFE9911895B7D7EA81FB816627772783
:1007020073D6A1EEBAE78BE392E4F6D634D68F0124
:1007120066247724E0E0E2BF60167106E8F3AAD708
:100722001AC51EDEE1E0EA93E2E0EA9339DEE2E096
:10073200EA93E2EFF1E0FA93EA9324DFE7E0EA9347
:10074200E2E0EA932DDEE1E0EA93E6EFF1E0FA93EC
:10075200EA9318DFE4E0EA93E3E0EA9321DEE1E0E2
:10076200EA93ECEFF1E0FA93EA930CDF2EDF0895BF
:100772007AD700E010E0E0E0EDBDECBD5524E7E003
:10078200EEBD7894E8EEF3E0FA93EA93B4DFE0E0AA
:10079200EEBDF894ECB5F0E0DF01EDB5FE2FE0E040
:1007A200EA0FFB1F8F01E52DFF2766277727AFEFA3
:1007B200BFEF80E090E00CD5DF01CB01F8016627A6
:1007C2007727E2D45AD708951A9310E010E018322E
:1007D20060F4E5E0F0E0FA93EA93CAD4879B02C0A2
:1007E200869901C01EE61F5FF2CF1991089567979F
:1007F200E0E0E883E983EA83EB83EC83ED83EE8335
:10080200EF835DDD75DD8DDFA0E0B0E054D5E03033
:1008120009F093C1909A9198D7DFAADFE3D5EC83D0
:10082200FD836E837F839098CFDFA2DFDBD5E883E1
:10083200F9836A837B83AC81BD818E819F81E0E0F5
:10084200F0E06AE774E4A6D6E887F9876A877B87CF
:10085200A0E0B0E280EA95E49DD6E887F9876A874E
:100862007B87A885B9858A859B8546D6EC83FD83DF
:100872006E837F83A881B9818A819B81E0E0F0E069
:100882006AE774E487D6E887F9876A877B87A0E0FE
:10089200B0E280EA95E47ED6E887F9876A877B87AB
:1008A200A885B9858A859B8527D6E883F9836A83DB
:1008B2007B83AC81BD818E819F81C9D5E887F98711
:1008C2006A877B87EC87FD876E877F87A1E0B0E030
:1008D200EAD4A885B9858A859B85A1D609F008F452
:1008E2000EC0A1E0B0E0DFD4A885B9858A859B85DA
:1008F200CDD4ADD5E887F9876A877B8705C0E0E06C
:10090200E887E987EA87EB87E1E0EA93E6E0EA93A2
:1009120047DDE2E0EA93E8E0F2E0FA93EA9332DEBE
:10092200A885B9858A859B85E8E2FBE66EEE7DE4C3
:1009320076D608F0F5C0E0EFF3E264E779E46FD62B
:1009420009F008F40DC0E0E0F4E264E779E422D6AD
:1009520098D4E2E0EA93FE017596FA93EA93A9D25B
:10096200A885B9858A859B85E0E0FCE36CE176E4A5
:1009720056D609F008F406C0E0EFF3E264E779E442
:100982004ED608F011C0A885B9858A859B85E0E01E
:10099200F0E06AE774E4FED574D4E2E0EA93FE0183
:1009A2007596FA93EA9385D2A885B9858A859B853F
:1009B200E0E0F0EC69E774E432D609F008F406C02E
:1009C200E0E0FCE36CE176E42AD608F00CC0E885AE
:1009D200F9856A857B8555D4E1E0EA93FE01759637
:1009E200FA93EA9366D2A885B9858A859B85E0E069
:1009F200F0E066EC72E413D609F008F406C0E0E019
:100A0200F0EC69E774E40BD608F00CC0E885F985D0
:100A12006A857B8536D4E2E0EA93FE017596FA9305
:100A2200EA9347D2A885B9858A859B85E0E0F0E004
:100A320060E070E4F4D509F008F406C0E0E0F0E00C
:100A420066EC72E4ECD508F00CC0E885F9856A859D
:100A52007B8517D4E3E0EA93FE017596FA93EA9355
:100A620028D2A885B9858A859B85E0E0F0E060E020
:100A720070E4D5D511F008F00DC0E0E0F0E06AE7CF
:100A820074E43AD5FED3E1E0EA93FE017596FA9357
:100A9200EA930FD2E1E0EA93E6E0EA9381DCE2E056
:100AA200EA93FE017196FA93EA937EDDEDE0EA9312
:100AB200E6E0EA9375DCA885B9858A859B85E0E046
:100AC200F0E060E070E4ABD528F4E1E0EA93EFE017
:100AD200F2E022C0A885B9858A859B85E0E0FCE327
:100AE2006CE176E49CD528F4E1E0EA93E2E1F2E0FD
:100AF20013C0A885B9858A859B85E0EFF3E264E798
:100B020079E48DD528F4E1E0EA93E5E1F2E004C06E
:100B1200E1E0EA93E8E1F2E0FA93EA9333DD0CC014
:100B2200E1E0EA93E6E0EA933BDCE2E0EA93EBE120
:100B3200F2E0FA93EA9326DD4DC1A0E0B0E0BBD328
:100B4200E13009F015C1909A91983EDE11DE4AD447
:100B5200EC83FD836E837F83909A919A35DE08DE63
:100B620041D4E883F9836A837B83AC81BD818E8122
:100B72009F8110D5E887F9876A877B87A885B98521
:100B82008A859B85B9D4E887F9876A877B87A88598
:100B9200B9858A859B85E0E0F0E060E87FE3ACD42C
:100BA200E887F9876A877B87A885B9858A859B85C7
:100BB200E0E0F0E060E87FE369D349D4E887F987B1
:100BC2006A877B87EC87FD876E877F87A885B985D3
:100BD2008A859B85E0E0FCE36CE176E420D509F0B0
:100BE20008F404C0E887F9876A877B87A5E0B0E04C
:100BF2005AD3A885B9858A859B8511D509F008F451
:100C02000EC0A5E0B0E04FD3A885B9858A859B8543
:100C12003DD31DD4E887F9876A877B8705C0E0E06A
:100C2200E887E987EA87EB87E1E0EA93E6E0EA937F
:100C3200B7DBE2E0EA93E8E0F2E0FA93EA93A2DCBF
:100C4200A885B9858A859B85E0E0F0EC69E774E4C4
:100C5200E6D409F008F40CC0E885F9856A857B853D
:100C620010D3E1E0EA93FE017596FA93EA9321D15B
:100C7200A885B9858A859B85E0E0F0E066EC72E4A0
:100C8200CED409F008F406C0E0E0F0EC69E774E4C1
:100C9200C6D408F00CC0E885F9856A857B85F1D257
:100CA200E2E0EA93FE017596FA93EA9302D1A885EF
:100CB200B9858A859B85E0E0F0E060E070E4AFD41E
:100CC20009F008F406C0E0E0F0E066EC72E4A7D4B4
:100CD20008F00CC0E885F9856A857B85D2D2E3E00D
:100CE200EA93FE017596FA93EA93E3D0A885B98553
:100CF2008A859B85E0E0F0E060E070E490D468F4DF
:100D0200E0E0F0E06AE774E4F7D3BBD2E1E0EA9313
:100D1200FE017596FA93EA93CCD0E1E0EA93E6E01D
:100D2200EA933EDBE2E0EA93FE017196FA93EA93DC
:100D32003BDCEDE0EA93E6E0EA9332DBA885B98595
:100D42008A859B85E0E0F0E060E070E468D409F019
:100D520008F405C0E1E0EA93E3E2F2E004C0E1E076
:100D6200EA93E6E2F2E0FA93EA930CDC2EDC32C07C
:100D7200E1E0EA93E6E0EA9313DBE2E0EA93E8E0FB
:100D8200F2E0FA93EA93FEDBF3DC2CD3E887F987EF
:100D92006A877B8776D2E0E0EA93FE017596FA9342
:100DA200EA9387D0E1E0EA93E6E0EA93F9DAE2E057
:100DB200EA93FE017196FA93EA93F6DBEDE0EA9389
:100DC200E6E0EA93EDDAE1E0EA93E9E2F2E0FA93AF
:100DD200EA93D8DBFADB879939C0C2DAE1E0EA9319
:100DE200E4E0EA93DDDAA0E0B0E065D2EF5F7FD223
:100DF200E33021F4A0E0B0E0E0E079D2A0E0B0E09E
:100E02005AD2E03031F4909AE2E0EA93ECE2F2E076
:100E120011C0A0E0B0E04FD2E13031F49098E2E0AE
:100E2200EA93E4E3F2E006C090989198E2E0EA9354
:100E3200ECE3F2E0FA93EA93A5DBC7DBE8EEF3E03A
:100E4200FA93EA9395D1879BFECF6BDC869905C016
:100E5200A0E0B0E030D2E23009F429C0A0E0B0E076
:100E62002AD2E03039F4EC85FD856E857F85A1E0DC
:100E7200B0E006C0EC85FD856E857F85A5E0B0E01B
:100E820026D26EDAE1E0EA93E4E0EA9389DAE2E07C
:100E9200EA93E4E4F2E0FA93EA9374DB96DBE8EE99
:100EA200F3E0FA93EA9364D1879BFECF3ADCACCCB1
:100EB200FFCF2497E0E0E883E983EA83EFE3EB8363
:100EC200D2D3EB85FC85EF3FAFEFFA0751F4EE8109
:100ED200FF81FA93EA93EEE4F2E0FA93EA933DD1CA
:100EE200EDC0EF3FAFE7FA0751F4EE81FF81FA93CD
:100EF200EA93EFE4F2E0FA93EA932FD1DFC0AC85F4
:100F0200AA238AF4E985FA856B857C8501D2E98773
:100F1200FA876B877C87AE81BF811196AE83BF83D0
:100F22001197EDE2EC93A885A73010F0E6E0E88790
:100F32001885E12F1150E03071F0AA81BB818C81BC
:100F42009D81EDECFCEC6CEC7DE3D6D2EA83FB8375
:100F52006C837D83EECFEA81FB816C817D81A985E3
:100F6200BA858B859C857AD2E987FA876B877C87DD
:100F720010E0E0E0F0E060E87FE3EA83FB836C836B
:100F82007D83EA81FB816C817D81A985BA858B8510
:100F92009C8545D378F0AA81BB818C819D81E0E05C
:100FA200F0E060E271E4A8D2EA83FB836C837D8384
:100FB2001F5FE7CF103049F4AE81BF811196AE8337
:100FC200BF831197E0E3EC933DC0E12F1150E03075
:100FD200C9F1AA81BB818C819D81EDECFCEC6CECAA
:100FE2007DE38AD2A0E0B0E080E09FE337D249D12E
:100FF20097D0EA83FB836C837D83A985BA858B8531
:101002009C85C8D2B8D10E2FAE81BF811196AE8316
:10101200BF831197E02FE05DEC93E02FAA81BB81A3
:101022008C819D81FF2766277727DED165D2A9852E
:10103200BA858B859C852AD10AD2E987FA876B8784
:101042007C87C3CFE885E030A9F1AE81BF811196DC
:10105200AE83BF831197EEE2EC93E885E150E88717
:10106200EF5F41F1A985BA858B859C85E0E0F0E0D0
:1010720060E271E441D2E987FA876B877C877BD192
:101082000E2FAE81BF811196AE83BF831197E02FE1
:10109200E05DEC93E02FA985BA858B859C85FF27BF
:1010A20066277727A1D1F2D0D2D1E987FA876B8759
:1010B2007C87D3CFAE81BF81E0E0EC93DBD22D966B
:1010C20008957B816A81F981E88177FB770F67FD5B
:1010D2007160972F9E5781F078F0983190F4AA278B
:1010E200BB27882708948795B795A7959A95D1F736
:1010F200EA23FB23682305C0E8947727EE27FF271E
:1011020066276F77769508F4606877F9A991B991A7
:1011120089919991EA17FB076807790797FB089568
:10112200E881F9816A817B81ACD0CBDFE883F983E6
:101132006A837B8329F4E881F9816A817B810BC010
:10114200D6F7A881B9818A819B81E0E0F0E060E86E
:101152007FE39CD07CD124960895E991F991A991DD
:10116200B991CD0105900D920020E1F7FC0108959F
:10117200E991F991309639F088EB9BE00197F1F70C
:10118200A8953197C9F70895EA0FFB1F681F791FC9
:101192000895F195E195F0400895F0956095709568
:1011A200E195FF4F6F4F7F4F0895FE2FFF0FFF0B0B
:1011B2006F2F7F2F08956F2F660F660B762F08957E
:1011C200FA9FF02DEB9FF00DEA9FE02DF10D0895AF
:1011D2007A9F702D6B9F700DF89F700DE99F700DB7
:1011E2006A9F602D710DFB9F600D711DE89F600D60
:1011F200711D8827FA9FF02D610D781FEB9FF00D6E
:10120200611D781FEA9FE02DF10D681F781F089578
:101212002AD0D6DF0EF4BDDF08950024112490E118
:10122200AA0FBB1F001C111C0E1A1F0A18F40E0E67
:101232001F1E01C0A1609A9599F7FD01D001089582
:1012420012D0EBDF0EF4A5DF0895E894B7FF04C0D7
:10125200A095B09511966894F7FD9BDFDEDFFD0146
:101262000EF497DF0895E894F7FF02C092DF6894C6
:10127200B7FF06C0A095B095119600F8039400FA46
:1012820008957A936A93FA93EA930895182E862F13
:10129200612D192E972F712D1B2EBF2FF12D1A2E76
:1012A200AE2FE12D0895129602D0BF01129711962A
:1012B20002D0FE2F1197E199FECFFF93FFB7F8946A
:1012C200AEBBBFBBE09AEDB3FFBFFF91089507D05D
:1012D20012960F01FB0103D0F0011297089507D077
:1012E2001196EF93EF2F03D0EF9111970895E19BA1
:1012F20002C0A895FCCF9FB7F894AEBBBFBBE09AE3
:101302008DB3E81719F0EDBBE29AE19A9FBF0895F9
:1013120030976040704009F070580895552342F4A8
:10132200503811F4E0FF04C03196691F791F6BF049
:1013320050E8572711F45F93CDC05F3F31F0660F3D
:10134200000C57956795752F08955F9300200AF05A
:10135200CDC0C6C050E8192E1522880F991F9527B7
:10136200550F879550E8072E0522660F771F7527C0
:10137200550F67950895689401C0E8945F93F2DF72
:10138200703818F07F3F08F4A5C056E1571BAAF445
:10139200519558300EF4593030F0EFEFFFEF6FEF08
:1013A2007FE777F91AC077275523B9F0EE0FFF1FB1
:1013B200661F771F5A95D1F710C07727583028F04B
:1013C200EF2FF62F672F5850F9CF552331F076952E
:1013D2006795F795E7955A95D1F700200AF4DDDE77
:1013E2005F910895689401C0E8943097604070401E
:1013F200B1F0002426F0772312F40094CEDE172EEB
:101402007EE1112032F07A95EE0FFF1F661F111C4C
:10141200F9CFEF2FF62F612D5F938ADF5F91089549
:101422004F93AF01FD01DA01AB01BC01CA01402DAE
:10143200012C142E4F910895EA0FFB1F681F089587
:10144200E095F0956095EF5FFF4F6F4F08955F93C2
:1014520081DF903871F150E8152604C05F937ADF7E
:10146200903839F1703821F1572F591B13F112F4CA
:10147200D7DFFACF583118F0AA27BB278827583070
:1014820028F0AB2FB82F88275850F9CF552329F0D1
:101492008695B795A7955A95D9F7502D512562F0A3
:1014A200CBDF38F46795F795E795739513F41EC073
:1014B200B7DF3EDF5F910895EA1BFB0B680B51F02B
:1014C20010F40094BDDF6623A2F3EE0FFF1F661F28
:1014D2007A95CBF7EE27FF27662777275F91089546
:1014E200EFEFFFEF6FE77FEF5F910895EFEFFFEF11
:1014F2006FE77FE75F9108955F932CDF703851F3B8
:10150200903841F301240894791F23F41CF300203E
:101512003AF3ECCF0F921F932F933F934F931127E0
:1015220022279927689FA0018F9F302D410D591FB7
:101532006B9F300D411D591F8E9F27D0BF9F25D015
:101542006A9F23D0BE9F1DD0AF9F1BD0AE9F110DAF
:10155200291F391F491F591FE32FF42F652F522FBF
:101562004F913F912F911F910F9066232AF0550FB3
:10157200EE1FFF1F661F02C073954BF2CFDE5F9115
:101582000895100D211D391F02C0200D311D491F64
:10159200591F08955F93DEDE703821F411200AF49A
:1015A2009FCFA4CF903809F495CF01240894970BCC
:1015B2001BF4D4F30020F3CF792F1F932F933F9383
:1015C2004F9311241127222733274427552790E2CE
:1015D200AE17BF078607410730F0AE1BBF0B860B65
:1015E200410B089401C08894551F221F331F111C00
:1015F200AA1FBB1F881F441F9A9551F7F901612D3D
:101602004F913F912F911F91662332F0550FEE1F9C
:10161200FF1F661F7A9543F281DE5F910895992339
:101622009AF0772342F0971748F029F4AE17BF07D4
:10163200860720F031F0989488940895989408943D
:1016420008951894889408957723C2F7971798F30A
:10165200A9F7EA17FB07680788F399F3ECCF5A93C7
:101662004A933A932A931A930A9308955D814C817F
:101672003B812A8119810881089509911991089560
:00000001FF
